:020000020000FC
:100000000C942D0A0C942A000C942A000C942A00BB
:100010000C942A000C942A000C942A000C942A00B8
:100020000C942A000C942A000C942A060C942A00A2
:100030000C942A000C942A000C942A000C942A0098
:100040000C942A000C942A000C942A000C942A0088
:100050000C942A0018959198899A0895919A899AF2
:080060000895919BFBCFF7CF3F
:1002000085BAE991F72F85BA649185BAE62FF1E0B6
:10021000000085BA0000099485BAE991F72F85BAE4
:10022000649185BAE62FF1E0000075BA00000994E8
:1002300085BAE991F72F85BA649175BAE62FF1E096
:10024000000085BA0000099485BAE991F72F85BAB4
:10025000649175BAE62FF1E0000075BA00000994C8
:1002600085BAE991F72F75BA649185BAE62FF1E066
:10027000000085BA0000099485BAE991F72F75BA94
:10028000649185BAE62FF1E0000075BA0000099488
:1002900085BAE991F72F75BA649175BAE62FF1E046
:1002A000000085BA0000099485BAE991F72F75BA64
:1002B000649175BAE62FF1E0000075BA0000099468
:1002C00075BAE991F72F85BA649185BAE62FF1E006
:1002D000000085BA0000099475BAE991F72F85BA34
:1002E000649185BAE62FF1E0000075BA0000099428
:1002F00075BAE991F72F85BA649175BAE62FF1E0E6
:10030000000085BA0000099475BAE991F72F85BA03
:10031000649175BAE62FF1E0000075BA0000099407
:1003200075BAE991F72F75BA649185BAE62FF1E0B5
:10033000000085BA0000099475BAE991F72F75BAE3
:10034000649185BAE62FF1E0000075BA00000994C7
:1003500075BAE991F72F75BA649175BAE62FF1E095
:10036000000085BA0000099475BAE991F72F75BAB3
:10037000649175BAE62FF1E0000075BA00000994A7
:1003800095BA0C94FE0685BA782487247824000058
:100390000000E991F72F6491E62FF1E0099475BA16
:1003A00078248724782400000000E991F72F6491D5
:1003B000E62FF1E0099485BA7424472474240000E0
:1003C0000000E991F72F6491E62FF1E0099485BAD6
:1003D00075245724752400000000E991F72F6491DB
:1003E000E62FF1E0099485BA76246724762400008C
:0E03F0000000E991F72F6491E62FF1E00994E7
:10040000000000000000000000F3E7DB0000C3CFA5
:10041000009024B4009024B4009024B4009024B43C
:1004200000000000000000000000000000000000CC
:1004300000000000000000000000000000000000BC
:1004400000000000000000000000000000000000AC
:10045000000000000000000000000000000000009C
:10046000000000000000000000000000000000008C
:10047000000000000000000000000000000000C0BC
:1004800000000000303030300000000030303030EC
:10049000000000000000000000000000000000005C
:1004A000000000000000000000000000000000004C
:1004B000000000000000000000000000000000003C
:1004C000000000000000000000000000000000002C
:1004D000000000000000000000000000000000001C
:1004E000000000000000000000000000000000000C
:1004F00000000000000000000000000000000000FC
:10050000000000000000000000F3E7DB0000C3CFA4
:10051000009024B4009024B4009024B4009024B43B
:10052000003078783078303030300000000000182B
:100530003030909060A830A830300000000000906B
:100540003030904890A8A84878A8A878607878308B
:1005500090309048A87878787878A84860903000F3
:10056000300060001800180060303060900000001B
:10057000000000003000000000000018306048C09B
:1005800000000000303030300000000030303030EB
:10059000000000000000000000000000000000005B
:1005A000000000000000000000000000000000004B
:1005B000000000000000000000000000000000003B
:1005C000000000000000000000000000000000002B
:1005D000000000000000000000000000000000001B
:1005E000000000000000000000000000000000000B
:1005F00000000000000000000000000000000000FB
:10060000000000000000000000F3E7DB0000C3CFA3
:10061000009024B4009024B4009024B4009024B43A
:100620000030787848187860601830300000001882
:100630007890181878606018787830301800601852
:1006400078787860786060607830307860A8A878D2
:1006500078787860307878787878183060307800FA
:1006600018006000180030006000006030000000DA
:10067000000000003000000000000030303090C06A
:1006800000000000303030300000000030303030EA
:10069000000000000000000000000000000000005A
:1006A000000000000000000000000000000000004A
:1006B000000000000000000000000000000000003A
:1006C000000000000000000000000000000000002A
:1006D000000000000000000000000000000000001A
:1006E000000000000000000000000000000000000A
:1006F00000000000000000000000000000000000FA
:10070000000000000000000000F3E7DB0000C3CFA2
:10071000009024B4009024B4009024B4009024B439
:10072000003000A8903030006018A8300000003081
:1007300078301830789090183078303030A83030D9
:10074000A878906078906060A830309060A8A87811
:100750007878783030787878307830303030000001
:10076000004890484830A848909090783090903059
:1007700090489048A87878787878A830303000C0D1
:10078000005490B4305490B4305490B4305490B479
:100790000000000000000000000000000000000059
:1007A0000000000000000000000000000000000049
:1007B0000000000000000000000000000000000039
:1007C0000000000000000000000000000000000029
:1007D0000000000000000000000000000000000019
:1007E0000000000000000000000000000000000009
:1007F00000000000000000000000000000000000F9
:10080000000000000000000000F3E7DB0000C3CFA1
:10081000000000009090909024242424B4B4B4B438
:100820000030007830307800601830A800A8003020
:1008300078303018A81878307848000060001830F8
:10084000A8A8786078609078783030906078A87840
:1008500090789018307878A8303030303030000000
:1008600000787860787830787830309030A8787870
:10087000787878603078787830783060301800C0D8
:10088000005490B4305490B4305490B4305490B478
:100890000000000000000000000000000000000058
:1008A0000000000000000000000000000000000048
:1008B0000000000000000000000000000000000038
:1008C0000000000000000000000000000000000028
:1008D0000000000000000000000000000000000018
:1008E0000000000000000000000000000000000008
:1008F00000000000000000000000000000000000F8
:10090000000000000000000000F3E7DB0000C3CFA0
:10091000000000009090909024242424B4B4B4B437
:10092000000000A8486078006018A83030003060EF
:1009300078306018181878607818303030A8300097
:100940006078786078606078783030786078A878FF
:1009500060A89018307830A87830603018300000E7
:1009600000787860789030487830309030A8787887
:1009700090486048307830A830486030303000C04F
:1009800000000000000000003030303030303030E7
:100990000000000000000000000000000000000057
:1009A0000000000000000000000000000000000047
:1009B0000000000000000000000000000000000037
:1009C0000000000000000000000000000000000027
:1009D0000000000000000000000000000000000017
:1009E0000000000000000000000000000000000007
:1009F00000000000000000000000000000000000F7
:100A0000000000000000000000F3E7DB0000C3CF9F
:100A1000000000009090909024242424B4B4B4B436
:100A2000003000789078480030303030300030604E
:100A300030A8A89018903060303030301800603006
:100A40004878904890A8604878A86078A87878306E
:100A500060487890303030787830A848189000009E
:100A6000004890484848301878A83078A8A87830CE
:100A700060186090184830A87818A830303000C04E
:100A800000000000000000003030303030303030E6
:100A90000000000000000000000000000000000056
:100AA0000000000000000000000000000000000046
:100AB0000000000000000000000000000000000036
:100AC0000000000000000000000000000000000026
:100AD0000000000000000000000000000000000016
:100AE0000000000000000000000000000000000006
:100AF00000000000000000000000000000000000F6
:100B0000000000000000000000F3E7DBC3CFC3CF0C
:100B1000000000009090909024242424B4B4B4B435
:100B200000000078300000000000000060000000BD
:100B30000000000000000000000000600000000055
:100B400000000000000000000000000000000000A5
:100B5000000000000000000000000000000000A8ED
:100B60000000000000000090000060000000000095
:100B7000601800000000000000900018006000C035
:100B800000000000000000003030303030303030E5
:100B90000000000000000000000000000000000055
:100BA0000000000000000000000000000000000045
:100BB0000000000000000000000000000000000035
:100BC0000000000000000000000000000000000025
:100BD0000000000000000000000000000000000015
:100BE0000000000000000000000000000000000005
:100BF00000000000000000000000000000000000F5
:100C00000F730D9308950D9108950F3709F40EE2B7
:100C10000D9308950D9108953F934F93A0E6B0E092
:100C20003EE103E0EDDF0BE1EBDF0FE0E9DF0FE397
:100C3000E7DF0CE3E5DF4EE10EE2E7DF4A95E1F79F
:100C40000FE70D933A9569F74F913F9108956A9593
:100C5000F1F708956FB76F93BF93AF93DF93CF937F
:100C6000FF93EF93000062B7623001F000000000D4
:100C70000000000062B7633001F0000000000000D7
:100C8000000062B7643001F0E601F70109947F01CA
:100C90006E0162E068BFEF91FF91CF91DF91AF915C
:100CA000BF916F916FBF1895F8946FB76F93BF9313
:100CB000AF93DF93CF93FF93EF9360E062BF6AE45B
:100CC0006CBF6AE063BF62E069BF0CC0AE98AF98CA
:100CD000A69AA79A979A8F980895AE9A67E0B7DF79
:100CE000AE98089587996CE0879B6CE0B62E6FEF05
:100CF000A62EF3DFEDE7F6E0CACF62E0A8DF000042
:100D0000BA9449F00000000000000000000000005C
:100D100000000000EECF87996DE0879B6DE0B62E56
:100D20006EEFA62EAF9AD9DFE7E9F6E0B0CF62E02A
:100D30008EDF0000BA9449F00000000000000000BF
:100D40000000000000000000EECF879969E1879B5A
:100D500069E1B62E6DEFA62EAF98BFDFE1EBF6E0AE
:100D600096CF62E074DF0000BA94D1F0000000007A
:100D7000000000000000000000000000EECF0FEFB8
:100D8000A016F1F3A016F1F7089500E0902E95BAA1
:100D900004B30F6304BB969A8E98959A8D98089524
:100DA000C0E6D0E0879969E1879B6EE1A62E74E0EA
:100DB000BB2493DFB0FE11C0869B11C0888085994B
:100DC000892CA4966CE043DF0000000085BAEAEEAF
:100DD000F6E05DCF95BA0C94FE060000000067E0D7
:100DE00036DF000000008990799049905990699011
:100DF000E991F72F6491E62FF1E00994B09421F086
:100E0000A49763E024DFD5CF73957C3029F0A497B5
:100E100061E01DDF0000CCCFAA9429F4000000009F
:100E2000000000005FCF0000000000000000000094
:100E3000000000000000BBCFA8E9B4E0E0E2F0E071
:100E4000ED93FD93E0E0F0E0ED93FD930895FF91C5
:100E5000EF91EE0FFF1F8F939F93CF93DF938591B9
:100E60009591A8E9B4E0CD91DD91C817D90708F0B4
:100E7000EC01CD93DD9305910D93219761F00197DE
:100E8000D1F7DF91CF919F918F91E0FD3196F6954B
:100E9000E795099405910197E9F7F3CF8F939F9315
:100EA000E8E9F4E03296819191910C910F3721F0AD
:100EB0000191ABDE0197C9F79F918F9108953E3163
:100EC00060F4153050F4A0E6B0E024E2329FA00DAB
:100ED000B11DA10F20E0B21F93CE08953E31E8F777
:100EE0001530D8F7A0E6B0E024E2329FA00DB11D86
:100EF000A10F20E0B21F87CE3E3178F74E3168F760
:100F0000A5E6B0E024E2329FA00DB11DA40F20E0C1
:100F1000B21F7BCE3E3108F74E31F8F6A5E6B0E0C1
:100F200024E2329FA00DB11DA40F20E0B21FB6CF66
:100F3000F1DF339508954F9340E089DF28002020AA
:100F400020202020202020202020202020202020A1
:100F50002020202020202020202020202020202091
:100F6000202020202020E4DF4F91089570DF200012
:100F7000202122232425262728292A2B2C2D2E2FF9
:100F8000303132333435363738393A3B3C3D3E3FE9
:100F9000CFDF5DDF2000404142434445464748499A
:100FA0004A4B4C4D4E4F5051525354555657585929
:100FB0005A5B5C5D5E5FBCDF4ADF2000606162639C
:100FC0006465666768696A6B6C6D6E6F7071727369
:100FD0007475767778797A7B7C7D7E20A9DF089599
:100FE0004F93A9DFA8DFA7DF335044E0BFDF4F9165
:100FF000089500E010E063DF9ECF10E060DF00E0C6
:1010000011E05DDF3395089500E3F7DF0CE3F5DFD2
:101010000CE0F3DF0FE0F1DF03E0EFDF03E3EDDFF0
:101020003650089514DF17002D275F5F602D2E5F67
:101030005F2E2D275F5F602D2E5F5F2E2D275F00B7
:1010400077DF0895EFDFEEDFEDDFECDFEBDFEADFE8
:1010500008950FE151DF33950895FBDFFADFF9DFE3
:10106000F8DFF7DFF6DF0895F2DE1000101C1C1C1D
:101070001C1C1C1C1C1C1C1C1C1C1C1059DFE7DE2F
:1010800010001018141010101418101818101C103C
:1010900014104EDFDCDE100010191018101E141E84
:1010A000141A1A1A101A1A1043DFD1DE1000101089
:1010B0001515151A101A1012161A1A1A1B1038DFE5
:1010C000C6DE1000101310121012101011101110A3
:1010D000131212102DDFBBDE1000101313131313A5
:1010E0001313131313131313131022DF0895AADF1E
:1010F0003650495EB2DF36504F5FB6DF4851089533
:10110000A6DE280041546D65676133322041565296
:10111000207543202B20536F6674564741203D2095
:101120003430306C696E65203730487A01DF8FDEED
:10113000280031382E3433324D487A2C2033636CFA
:101140006B2F7069786C2C20347069786C2F636811
:1011500061722C20343063686172EADE78DE280028
:10116000347838706978656C20666F6E742C20391D
:10117000352041534349492C20313620626C6F633E
:101180006B67726170686963D3DE08950F9300E046
:1011900010E095DE0F910F9311E091DE0F910F9308
:1011A0000A7212E08CDE0F910F93057113E087DE57
:1011B0000F910A6214E083DE3395089503E0E6DFC1
:1011C0000CE0E4DF0FE0E2DF00E3E0DF03E3DEDF7B
:1011D0000CE3DCDF0FE3DADF3750089538DE280058
:1011E0006E6F720E696E760F6E6F720C756C696E33
:1011F0000D6E6F720B322F330B6E6F720A312F33FD
:101200000A6E6F720970617393DE0895E7DFE6DF9F
:10121000E5DFE4DFE3DFE2DFE1DF089518DE280049
:1012200064657369676E20616E6420636F64652016
:101230006F70656E20736F7572636520617661698A
:101240006C61626C6520617473DE01DE2800687475
:1012500074703A2F2F6E65696C2E6672616E6B6CBE
:10126000696E2E63682F50726F6A656374732F53B3
:101270006F66745647415CDE08953F934F9330E0AC
:1012800040E0AEDEB6DEC0DE32DFB3DE39DFB1DE37
:1012900095DFBCDFAEDEC2DFACDE4F913F9108953B
:1012A00010E01CDE005F0BDE0895949A8C98849900
:1012B0000895052F0F7341F43F9330E0F1DF33952C
:1012C000EFDF3395EDDF3F9108953F934F9336E184
:1012D0004091000030DE3150939A8B98839910C072
:1012E0004091BC04052F0F7031F443954E3108F046
:1012F00040E04093BC04ABDD04005F405F2F18DE8C
:101300004F913F910895A3DD06002020202020204A
:101310000FDE0895F8DFF7DFF6DFF5DFF4DFF3DF48
:10132000089595DD03002E2D2E0002DE90DD0300D2
:101330007C207C00FDDD8BDD0300602D2700F8DDC7
:10134000089585DD03002E2D1000F2DD80DD030001
:101350007C201500EDDD7BDD0300602D1000E8DD55
:10136000089575DD03002E1C1000E2DD70DD030022
:101370007C101500DDDD6BDD030060131000D8DD8F
:10138000089565DD0300101C1000D2DD60DD030050
:101390001A101500CDDD5BDD030010131000C8DD51
:1013A0000895123018F410FFBCCFCBCF10FFD9CF67
:1013B000E8CF3F934F9334E040E044DE3650929ABA
:1013C0008A9882991CC040E148DE36504395A2DFDE
:1013D0003650052F069506950695102F077027E0C5
:1013E00002FD201B02FD022F300F1695139517707A
:1013F00027E012FD211B12FD122F410FD2DF4F916A
:101400003F9108953F934F933BE040E079DE3350A6
:10141000919A8998819911C050FD0FC054FD0DC05B
:101420004091BD04052F0F7331F443954E3108F000
:1014300040E04093BD040FE55FDD4F913F9108957B
:101440001CDF50E05093BC045093BD0498DC5395CE
:101450002CDF3BDFAEDFD6DFF9CFEFE5F8E0EDBF05
:10146000FEBF7894D9DB32DC90DC1EDCE5DCE8CF13
:00000001FF
